:020000020000FC
:10000000E1C949C20000000025C000004FC1000046
:10001000000052C1000000000000000002030406BE
:10002000080C101820304060800002030406080C01
:10003000101820304080FF000406080C10182030F3
:10004000406080A0C0000D0D0405060D050D0603DF
:10005000030302004FB662FD1EC070FF1AC165FDAA
:10006000FAC00994C0919700C395C0939700C5E06A
:10007000C519B8F3D0919700CD1B98F3C8E7089441
:1000800083FDC795C4BDC52DCC2321F4C0E083FDFD
:10009000C0E8C4BD09C171FF03C0919890989398BE
:1000A000C52D089483FDC795C4BDC09399006B7F8F
:1000B000C52DCF3F09F443C0C0919800C395C093AC
:1000C000980070FF37C082FD05C091989098939872
:1000D0004FBE18957860C091A000CC2391F0C091DC
:1000E0009800CA95D091A000CD1B58F0777FC091A1
:1000F0009800D0919F00CD1B08F41CC0209298005E
:1001000019C0919890989398C5E0CA95F1F7C0915D
:100110007500CA95C2FD09C0C1FD05C095FF95983F
:1001200095FD94980EC097980CC095FF949895FDF6
:10013000959807C09198909893984FBE18952092E3
:1001400099004FBE1895A5C0552021F095FF919AB2
:1001500095FD939A90989DC0552009F0909A95FF2F
:10016000939895FD919895C0552021F095FF939A0D
:1001700095FD919A95FF919895FD93988AC095FF6A
:10018000949A95FD959A95FF959A95FD949AC5E058
:10019000CA95F1F7552021F095FF919A95FD939A14
:1001A000909877C095FF949A95FD959A979AC5E097
:1001B000CA95F1F7552021F095FF919A95FD939AF4
:1001C000909867C0979A95FF949A95FD959AC5E087
:1001D000CA95F1F7552009F0909A95FF939895FDEF
:1001E000919857C0979A95FF959A95FD949AC5E076
:1001F000CA95F1F7552009F0909A95FF939895FDCF
:10020000919847C095FF959A95FD949A979AC5E065
:10021000CA95F1F7552021F095FF939A95FD919A93
:1002200095FF919895FD939834C095FF959A95FD0B
:10023000949A95FF949A95FD959AC5E0CA95F1F721
:10024000552021F095FF939A95FD919A95FF9198ED
:1002500095FD93981EC082FF1CC0C0917500C2FD21
:100260000BC0C1FD11C095FF949A95FD959A95FF1D
:10027000959A95FD949A0DC0C1FDF5CF95FF949A7E
:1002800095FD959A979A05C0979A95FF959A95FD31
:10029000949AC52DC095089483FDC795C4BDC0939D
:1002A00099002092970064604FBE18954FB6C0E148
:1002B000C8BF6E7F4FBE18953FB68F7EABB7A07498
:1002C000A2118061A0E0ABBFA9B7AE7FA9BF7894AF
:1002D000A0916600AA2349F0A92FAF7151F1A09116
:1002E0006600AA95A093660024C040E050E0A0B349
:1002F00096FFA095A2FD4FEF96FDA3E096FFA2E02A
:10030000A5BFAA27A064AABF8D7FA0B396FFA09522
:10031000A2FD5FEF451749F7A8E161FDA0936600D4
:10032000A92FAF7119F0A8E1A093660040938D004A
:100330008160A0916700AA2331F0A0916700AA957F
:10034000A093670007C0A92FAF7121F08061AA2791
:10035000A064AABF80FF4BC0A0918D004A2F8E7F62
:10036000A92FAF71E1F0A091AE00A430C1F4403FDD
:1003700008F040EFA42FA295AF704A0F5091B00043
:10038000533069F0A695A69550FD01C0A69552FD83
:1003900003C0A41B4A2F03C04A0F08F44FEF409339
:1003A000610071FF08C0A091610050919200A517F3
:1003B00010F0509361004091AE00443029F5A091B7
:1003C000610040916300A41B70F04091CF00A40B2A
:1003D00050F0A0916300A40FA093630040F4AFEF2E
:1003E000A093630004C0A0916100A09363004091BA
:1003F0006300A09192004A1708F04A2FA091940040
:100400004A1708F04A2F542EA52DA03408F0686032
:10041000A0916000A395A093600051F0F894A9B753
:10042000A160A9BF84FF02C0A0E4ABBF3FBE189586
:1004300041E050916600552331F0A92FAF7119F4B6
:100440005A9550936600A0918D00A13018F020922B
:1004500090000DC02092910020929A00A0919000EF
:10046000AF5FA093900018F0AFEFA0939000A09121
:100470009300A65F20F05FEF5093930002C0A0931B
:100480009300F894A9B7A160A9BF84FF02C0A0E4BB
:10049000ABBF3FBE18953FB64CB55DB58F7EABB7D1
:1004A000A074A2118061A0E0ABBFA9B7AE7FA9BFC5
:1004B000789481FD26C096FDA2E096FFA3E0A5BF3B
:1004C0008260A0B396FFA095A2FF05C04093640090
:1004D0005093650033C196FDA3E096FFA2E0A5BF4F
:1004E000AA27A064AABF8D7FA92FAF7109F417C1F5
:1004F00040E0A0B396FFA095A2FD11C140938D00EE
:1005000004C196FDA3E096FFA2E0A5BF8D7F61FF29
:100510006BC096FDA2E096FFA3E0A5BFAA27A0644A
:10052000AABF82604093880050938900A090860003
:100530004A19B09087005B09BB24A2E0EA2EA22CE6
:10054000483CA0E05A0730F4A0E1BA2EE22CAAE021
:10055000AA2E27C04836A1E05A0730F4A8E0BA2EE8
:10056000E22CAFE0AA2E1DC0403DA2E05A0730F4B5
:10057000A4E0BA2EE22CAEE1AA2E13C0403AA5E0C8
:100580005A0730F4A2E0BA2EE22CACE3AA2E09C03E
:100590004839A8E05A0728F4A1E0BA2EE22CA8E7CF
:1005A000AA2EC42EA0918A00CA1AD52EA0918B0023
:1005B000DA0ADD202AF4AFEFC094D094CA1ADA0A1E
:1005C00020928C00CA14DE0418F4A1E0A0938C00E1
:1005D00040938A0050938B0040918800509189008D
:1005E0004093860050938700A09164004A1BA0911D
:1005F00065005A0B94FD7CC093FD7AC092FD76C0D5
:100600005695479591FD72C05695479590FD6EC0E1
:10061000D52EC42ED694C79461FD0CC0AC2DAC5120
:10062000AD2DA24008F07BC0DD2021F4AC2DA85CEC
:1006300008F475C0A0E0EA2E97FD08C0E090C20063
:10064000A091B400A33011F4E090CA00AAEFEA0E22
:10065000F22CF21CCE18DF084FB74170A091B40005
:10066000A330A9F4442329F095FD11C0F8949062B9
:1006700004C095FF0CC0F8949F7D91989098939832
:10068000949A979A959A71FD01C060687894442372
:1006900069F0A091B400A33031F4AFEFC094D094CE
:1006A000CA1ADA0A03C040E050E022C0A091B400A8
:1006B000A33049F4CC0CDD1CA5E0CA1AD20818F40A
:1006C000A0E0CA2ED22CAFEFCA16D20418F04FEF1A
:1006D00050E00EC0F090A700CF9C412D000C441FAD
:1006E00050E008F012C04FEF50E00FC0569547950C
:1006F00094FF07C0552309F04FEFA42FA6954A0F8A
:10070000521D4F3F520508F04FEF40938D0081601E
:1007100061FF05C0AFE1A095A923AB299A2FA8E1FD
:10072000A0936600A92FAF7119F4AAE0A093660008
:1007300061FD04C0A92FAF7109F08F7EA6E0A093E0
:100740006700A92FAF7119F4AAE0A0936700F8948D
:10075000A9B7A160A9BF84FF02C0A0E4ABBF3FBEA0
:10076000189511E00AC013E008C01AE006C01EE1A7
:1007700004C014E602C018EC00C005E1BB27BA951E
:10078000F1F70A95D9F71A95C1F708952AE338E7E2
:1007900009C020E33CE806C02AE234EB03C025E2AE
:1007A00038EC00C0652CB1E05B2E12E095FD9F7D1A
:1007B00095FF9062BB27979ABA95F1F7552009F0FB
:1007C000909ABA95F1F79098BA95F1F79798BA95EB
:1007D000F1F7552021F095FF919A95FD939AB091EC
:1007E000A800BA95F1F795FF919895FD9398B7E811
:1007F000BA95F1F71A95D1F6022FB22FBA95F1F703
:100800000A95D9F73A9571F6979A562C0895221BB6
:1008100039E0001F3A9509F40895221F211B18F4AE
:10082000210F8894F6CF0894F4CF622C722CB0E09C
:100830008894B395221F331FE0F737952795889446
:10084000912E802E020B130B10F4192D082D10F48D
:10085000889401C00894661C771CBA9571F7172D0F
:10086000062D0895322D11232AF43A9500951095FE
:10087000031B130BF894029F712C002D129F912CD7
:10088000802C7894780C172D921C292DB4E06B2EB7
:100890002695179507956A94D9F7332321F000958B
:1008A0001095031B130B08950091AE000430A1F1C5
:1008B000B0918D00B15008F010C0B0916100B093BC
:1008C0006300209277002092780020927900209295
:1008D0007A0020927B006F7B1FC06090AE00606446
:1008E000B0916100B093620008E317EC20917300AF
:1008F0003091740036952795B62DBA9541F036950E
:100900002795B62DBA95BA9511F0369527958DDFB6
:100910000093770010937800089566FF1BC0009144
:100920007700B09162000B1B10917800120928F437
:100930000038BFEF1B0740F009C00F37120508F45D
:1009400005C00FE710E002C000E81FEF00937C0035
:1009500010937D00089566FF39C000917C00B0912E
:1009600079000B0F10917D00B0917A001B1F20E0E1
:1009700030917D0033230AF42A95B0917B002B1F20
:100980001AF4203F40F00AC02F3008F407C00FEFE0
:100990001FEF2FE003C000E010E020EF3091630074
:1009A000B09192003B1718F4332331F009C0B09195
:1009B0007D00BB235AF004C0B0917D00BB2332F40C
:1009C0000093790010937A0020937B00089566FFCE
:1009D0002FC02091CD0000917C00000F10917D0070
:1009E000111F40DF11232AF40038BFEF1B0740F02E
:1009F00009C00F37120508F405C00FE710E002C068
:100A000000E81FEF002352F0B0916200B01B0B2FE3
:100A100018F0013008F00AC001E008C000950F5F2F
:100A2000B09162000B0F08F001C00FEF00937E0041
:100A3000089566FF2DC02091CE0000917A0010919C
:100A40007B0010DF11232AF40130BFEF1B0740F0B9
:100A500009C00F3F120508F405C00FEF10E002C0F7
:100A600001E01FEF112352F0B0917E00B01B0B2F5D
:100A700018F0013008F00AC000E008C000950F5FD0
:100A8000B0917E000B0F08F001C00FEF00936300E0
:100A900008950FEF677FB72FB670E9F46860B091E3
:100AA0007400B83008F0677FB0917400A1F00FEFC8
:100AB00010917400ACDEF894B09170000B9F112D72
:100AC000002D7894112309F00FEFB09195000B17CA
:100AD00010F40091950000939400089546D374FF9C
:100AE000B7E074FDB7E0B068B064B7B9B6B1B0684C
:100AF000B064B6B936DE74FFB7E074FDB7E0B06835
:100B0000B064B7B9B6B1B068B064B6B9B6B1B6FD45
:100B1000FDCF04B115B1B6B1BF77B6B979D32DE623
:100B20002093A30030E03093A400732E7694622EBD
:100B30006694620E731E262D372D0217130778F068
:100B40008090A300BDE6B80DB093A3008090A400F0
:100B5000B0E0B81DB093A400260D371DEECF8090F5
:100B6000A3009090A4001091A40016950091A300FA
:100B7000079516950795B091A300B00FB093A1000B
:100B8000B091A400B11FB093A20023E01695079581
:100B90002A95E1F72091AF002A9529F42092A3002D
:100BA0002092A4000AC02A9521F0800E911E2A9559
:100BB000E1F78092A3009092A40008952091AF00E5
:100BC000B6B1B6FDFBCF04B115B1B6B1BF77B6B9BA
:100BD000B091A500B395B093A500B83060F1209214
:100BE000A500B091CC00BB2321F1112329F0B091D5
:100BF000A600BF3F61F009C0B091A6000B1739F005
:100C000020F4BB2321F0BA9502C0B395E1F3009123
:100C10009200B093A600B03050F400ECB03038F43D
:100C200000E8B03020F400E4B03008F400E00093B5
:100C300092007F7E0895213099F00F3FB3E01B07AB
:100C400078F4B091A3000B17B091A4001B0740F4F7
:100C5000B0919200BB23A9F0BA95B093920011C055
:100C6000B0919200BF3F69F0B395B0939200B091FC
:100C7000B400B33031F4B0919200BC5F10F4B09383
:100C8000920000919200B0916300B01B10F40091AB
:100C90006300B09193000B1750F000919300B09156
:100CA0009300BF3F21F0B0919300B0939200B091B8
:100CB000AE00B43009F406C0B09194000B1708F0F0
:100CC0000B2F502EB091A500B73009F47061089534
:100CD00002E3F894B091D0000B9F012D000C001F8F
:100CE0007894B09192000B1710F00091920000934D
:100CF000610000936300502E0093950008952092A8
:100D00007300B8E0B0937400089520918000309192
:100D10008100F8940CB51DB5200F311F3BBD2ABDD5
:100D20006160B0E1B8BF7894209171003091720099
:100D30000093710010937200021B130B209173003B
:100D400030917400622E732EB4E08B2EB2E09B2E95
:100D5000B0917400B43010F08A949A94B83010F0C6
:100D60008A949A94769467948A94E1F726193709BD
:100D7000992021F0169507959A94E1F7200F311FDD
:100D8000209373003093740008F00895BFEFB09380
:100D90007300B09374000895209182003091830015
:100DA000F8940CB51DB5020F131F1BBD0ABD616081
:100DB000B0E1B8BF7894089560FDFECFEDDF0895EF
:100DC000B091BE0000916E00023808F0B395003A71
:100DD00008F0B395B63008F0B5E09B2EBCE08B2E42
:100DE000B0917400B33030F48394839482FF02C0D6
:100DF00083948394B23030F48394839482FF02C04E
:100E00008394839471FF03C0B3E09B2E822C1091D6
:100E100074000091730024E0169507952A95E1F778
:100E20000819120928F0B02FB250B12FB20910F4EE
:100E300002E010E0312F202F712E602E76946794FF
:100E4000B92DB330E9F0B0FD05C0060D171D262DF4
:100E5000372D06C0000F111F0250120922E030E0AA
:100E6000B92DB33068F0209384003093850000934F
:100E70008000109381006092820070928300089538
:100E800000938400109385002093800030938100AC
:100E90006092820070928300089560FDFECF2091E1
:100EA0008200220F30918300331FB72FB67021F0DC
:100EB0002091730030917400F8940CB51DB5020FA9
:100EC000131F1BBD0ABD6160B0E1B8BF78940895DF
:100ED00060612092760020E004C06061209276007C
:100EE00020E2B72FB67009F06F7E789460FD05C0E0
:100EF000B0917600BB2309F0089501E063FF0AC0BA
:100F0000B0917400B33008F002E0B0917400B630D4
:100F100008F003E071FF01C006E060FD06C0B0917B
:100F20007600BB2311F0789408951AE083FF1AE04D
:100F3000789400000000F89462FD03C014E183FF80
:100F400014E171FF01C018E7B4B530919900B31BEB
:100F5000B10B18F3B0917600B395B0937600B5E07D
:100F60003B2F6B2E722CB8B1B072B21709F073948C
:100F70003A95C9F77394761488F464FFB2CF6F7E04
:100F80003CB56DB47090730080907400370D681C90
:100F90006BBC3ABD6160B0E1B8BFA3CF64FDA1CF27
:100FA0000A9509F0BACF7894089571FF0AC0B091FC
:100FB0006D00B395B0936D0060FD0CC020926D0084
:100FC00009C060FD07C064FD05C067FD03C0BF9197
:100FD000BF91A5C408952091840030918500F894B4
:100FE0000CB51DB5020F131F1BBD0ABD6160B0E13A
:100FF000B8BF78940895EFDF00E063FF03C064FF9B
:1010000001C001E0F89410916E00B7E01B9F212D04
:10101000102D7894200F26951795269517952695CF
:10102000179510936E00183718F4B8E7B0936E0058
:1010300000916E00B0916F000B1720F060629198E4
:101040009098939860FDFECF0895F894949A979A9B
:10105000959A82FF07C0E2E0F1E073FF03C0BEE1B2
:10106000BA95F1F7B0917400BC7F81F0552021F062
:1010700095FF919A95FD939AB6E0BA95F1F795FF91
:10108000919895FD9398B5E0BA95F1F795FF9498EE
:1010900095FD9598B2E0B0937500ABC0F89495FFBC
:1010A000939895FD919882FF0DC0E2EFF0E073FFF9
:1010B0000BC0979A95FF959A95FD949ABEE1BA95C3
:1010C000F1F702C0ECEAF0E062FF03C0552009F03E
:1010D000909AB3E0B09375008CC0F894949A979A64
:1010E000959A82FF07C0E2EEF0E073FF03C0BEE115
:1010F000BA95F1F7B0917400BC7F81F0552021F0D2
:1011000095FF939A95FD919AB6E0BA95F1F795FF00
:10111000939895FD9198B5E0BA95F1F795FF95985C
:1011200095FD9498B4E0B093750063C0F8949098DE
:1011300082FF0DC0E2EDF0E073FF0BC095FF949AC3
:1011400095FD959A979ABEE1BA95F1F702C0E4EA47
:10115000F0E062FF06C0552021F095FF919A95FDC1
:10116000939AB5E0B093750044C0F894949A979A16
:10117000959A82FF07C0EFEBF0E073FF03C0BEE17A
:10118000BA95F1F7B0917400BC7F51F0552009F089
:10119000909AB6E0BA95F1F79098B5E0BA95F1F764
:1011A0009798B6E0B093750024C0F89495FF919895
:1011B00095FD939882FF10C0E5E1F1E073FF0EC04A
:1011C00095FF949A95FD959A95FF959A95FD949A19
:1011D000BEE1BA95F1F702C0E4EBF0E062FF06C0B1
:1011E000552021F095FF939A95FD919AB1E0B09327
:1011F000750067FF0AC00CD0BEE1BA95F1F7B5E003
:10120000BA95F1F79498979895986F7D789408958A
:1012100023EA30E0F901919890989398949A979ADC
:10122000959A6B7F0895ACEAB0E009E00D9309E070
:101230000D9304E00D9301E00D9303E00D930FEF88
:101240000D930AE00D9301E00D9301E00D9301E091
:101250000D93A8EBB0E001E00D930FEF0D930D930C
:101260000FEF0D930D930D9303E00D9306E00D9397
:101270000FEF0D930D9305E20D9300ED0D9308E232
:101280000D9300E50D9304E00D930DE00D9302E046
:101290000D9300E00D930AE70D930FEF0D9301E01E
:1012A0000D9308952091BF0009E011E0223011F460
:1012B00005E011E0233011F405E012E0243011F4D0
:1012C00005E013E0253011F409E017E0263011F4B1
:1012D00000E010E000939F001093A0002091B30065
:1012E0008B7F233009F48460777F233009F47860A2
:1012F000B091B400B33019F09F7DB1FD90629F7B37
:10130000B091B500B1FD9064B22FB23011F0886099
:1013100001C0877F0895ECE1F0E00091AC000A95F0
:10132000E00FF21DB491B093CD000091AD000A958D
:10133000E00FF21DB491B093CE006ADF0895EAE2A7
:10134000F0E00091C7000A95E00FF21DB491B09350
:10135000CF005EDF0895E8E3F0E00091B2000A9567
:10136000E00FF21DB491B093D00052DF08950895BC
:10137000B091C8000FEF1CE0B23011F400EA1AE09F
:10138000B33011F402E815E000936F001093700081
:10139000089508952091C2003091C30097FF02C0C4
:1013A00020E03FEFB32FB21B6B2EB25810F4B2E81F
:1013B0006B2E00E00395609EB12DB058D8F30093DA
:1013C000A7000895F894E3E0F0E0B9E0B7BFB49166
:1013D000B078C1F3F894A895B1B5B861B1BDB0E0EB
:1013E000B1BDB4E0BEBFBFE5BDBF12DFB0E0B8BB6A
:1013F000B0E1B7BBB0E0B5BBB0E0B4BBB0EBB2BBE3
:10140000BBEBB1BB2224A0E0B0E02D92AA31E9F7FA
:10141000A0E6B0E00FEF2D920A95E9F704DF9FD226
:1014200041DF79DF8CDF97DFA2DFA2DFB2DFB2DF3F
:101430000091C4000093A800EBDEB2E0B3BFB2E0BD
:10144000BEBDB2E0B5BDF89496D9A0D990D9A1D9C6
:101450008ED9A2D98CD98FD98ED98BD9B1E5B8BF05
:10146000B9BFB0B7B860B0BFB6B1B460B6B979D9DA
:10147000789434DBB0E4BBBFBB27B064BABF8D7FC8
:101480007AD9B1E0B0936900626025E0B0918C0038
:10149000BB2309F425E067D9B0918D00B230A8F3E1
:1014A000B92FBF7100918F0000938E00B0938F0011
:1014B000B01759F72A9551F76D7F96FDB3E096FF67
:1014C000B2E0B5BFBB27B064BABF8D7F52D94BD94C
:1014D00002E0B92FBF7109F400E0B0918D00B017A0
:1014E000B0F3F89453D952D951D9789444D9209271
:1014F0007F00B091B400B33009F472C034D9B09118
:10150000B800B13008F46CC0B0916900B13008F493
:1015100067C0B92FBF71C1F0B0918D00BF3F08F413
:101520005FC0F8943CD9789424D9B0918D00B13043
:10153000C0F7F8942BD919D929D978941AD9B09130
:101540008D00BF3FB0F3D4C2B3E09B2E9068F894F7
:1015500021DF78940ED9F8949F771CDF80908D005E
:10156000B0918D00BF37789408F442C0FAD8F8944F
:1015700016D978949A9451F7B82DB550B093C3000A
:10158000FAD8F89419D287D27894BAE09B2E906852
:10159000F89400DF7894EDD8F8949F77FBDE809084
:1015A0008D00B0918D00BF37789478F7DAD8F89431
:1015B000EDD8DBD8EBD878949A9449F7B82DBB5F77
:1015C000B093C200D8D8F894F7D174D27894D1D817
:1015D000F894E0DE7894B0918D00BF3FC0F388C2EC
:1015E00000918D00B0917F000B1710F000937F00E9
:1015F000C0D801E0B091B400B35009F405E0B09157
:101600008D00B01708F075CFF894C9D8C8D8C7D8DE
:101610007894B1D82092690020926A0020926B00E1
:10162000B0916A00B395B0936A00BF3F69F5B0917D
:101630006B00B395B0936B00B091C60009E1BA9509
:1016400059F002E3BA9541F00DE7BA9529F00AEF97
:10165000BA9511F020926B00B0916B00B017A0F01A
:10166000B0916B00BA95B0936B00B4EBB0936A0085
:10167000B091C500B093A800F89491D87894B09137
:10168000C400B093A80075D870D8B0916600BB2391
:1016900021F4B92FBF7109F4F7CEB0918D00B630A7
:1016A00008F4BECFB091B400B35009F062D8B09145
:1016B0006600BB2309F4E8CEF894AADD209261000D
:1016C0002092620020926300522C7894B091B10075
:1016D000B0939600209277002092780020927900B3
:1016E00020927A0020927B002092A50060E070E0BA
:1016F00020926E0004DBB8E0B093A500706131D891
:1017000074FFB7E074FDB7E0B068B064B7B9B6B1C4
:10171000B068B064B6B9B6B1B6FDFDCF04B115B1CD
:10172000B6B1BF77B6B9112309F00FEF0093A60049
:1017300045DAB8E0B093A50070618090B300B2E0E4
:10174000B093B300AFDD8092B300F894BFEFB093D5
:101750009200BEDAB0916100B0939200B093930012
:10176000B09394007894B1E0B0936100B0936300BB
:101770005B2EB0939B00B0919100B0939A00716082
:10178000726020926D00F1DC10DDBFDAB8DA18DB90
:1017900004C088DD2092A5007F7E95FFB2E095FD14
:1017A000B4E0B068B064B7B998DBFFDB14DC7CD878
:1017B00022DC4BDCAADA00DB03DB6FDBB3E0B068D2
:1017C000B064B7B985DBF1DB06DCA7D862D913DCDE
:1017D00065DC9BDAF1DAF4DA60DB95FFB4E095FDC5
:1017E000B2E0B068B064B7B978DBDFDBF4DBB3D864
:1017F00002DC73DC8ADAE0DAE3DA4FDB95FFB2E091
:1018000095FDB4E0B068B064B7B962DBCEDBE3DB72
:10181000DED8F1DB8BDC79DACFDAD2DA3EDBB3E08B
:10182000B068B064B7B959DBC0DBD5DB02D9E3DB04
:101830009CDC6BDAC1DAC4DA30DB95FFB4E095FDED
:10184000B2E0B068B064B7B943DB74FFB7E074FDD1
:10185000B7E0B068B064B7B9B6B1B068B064B6B953
:10186000A4DBB9DBC8DBA1DC50DAA6DAA9DAA6D999
:1018700014DB71FF2EC067FD2CC0B0919500B093B2
:101880009200B0939300B0919100B0939A00B1E0B0
:10189000B0939B0014E624E1B0916D00B11798F06D
:1018A0007D7F746020936C00B091B400B33051F42C
:1018B000B0919500B0939200BFEFB0939300B0E267
:1018C000B093940006C0B0918D00B13008F065CFA0
:1018D00026C072FF10C067FD0EC0B0916C00BA95B3
:1018E00011F47B7F56CFB0936C00B0918D00B13076
:1018F00008F053CF14C0B0919000BA3F80F4B92FD4
:10190000BF7121F4B0916600BB2349F0B09174001F
:1019100000EF67FF01C000E6B01708F43ECFF8946F
:1019200077DC8090B300B2E0B093B300BBDC809270
:10193000B300209261002092620020926300522C3A
:10194000209296007E7F78940CD762DCB92FBF710D
:1019500029F4B0916600BB2309F496CD5DCEEDE08D
:10196000F0E023D0053509F01BC0EEE0F0E01DD01B
:101970000A3A09F015C03AE0ACEAB0E0E3E0F0E082
:1019800014D00D9331963A95D9F735E1A8EBB0E034
:10199000EFE0F0E00AD00D9331963A95D9F702C006
:1019A00042DC0AD0E4E2F0E00895E199FECFEEBB1C
:1019B000FFBBE09A0DB308951ED03AE0ACEAB0E068
:1019C000E3E0F0E00D910FD031963A95D9F735E18B
:1019D000A8EBB0E0EFE0F0E00D9105D031963A953C
:1019E000D9F712D00895E199FECF0DBBEEBBFFBB36
:1019F000E29AE19A0895EDE0F0E00FEFF4DFEEE017
:101A0000F0E00FEFF0DF0895EDE0F0E005E5EBDF4B
:101A1000EEE0F0E00AEAE7DF08953091A9000091D6
:101A2000AA00313011F40093AC00323011F400936D
:101A3000AD00333011F40093AE00343011F4009354
:101A4000B000353011F40093AF00363011F400933C
:101A5000B200373011F40093BE00383011F4009317
:101A6000C700393011F40093BF003A3011F40093ED
:101A7000B3003B3011F40093C8003C3011F40093E4
:101A8000B4003D3011F40093B500089525E073D6FD
:101A90002A95E9F708957AD67CD67ED680D665D683
:101AA00075D677D679D67BD660D670D672D674D6F0
:101AB00076D6089574D670D66CD668D656D66FD6BC
:101AC0006BD667D663D651D66AD666D662D65ED650
:101AD00008958090A9009090AA0058D657D656D65F
:101AE00044D68A94D1F75BD640D69A94E1F708950C
:101AF000F894D1DF7894CADFC9DFB1E0B093A900D0
:101B0000B1E0B093AA002092AB00F894E2DF7894A1
:101B1000B5E06B2E70908D002ED6B0918D007B16A7
:101B2000C9F7B13018F0BF3F40F107C076DFF89435
:101B300043DFB1DFB8E0B1BDA9DF6A9459F7B091D6
:101B4000AB00B395B093AB00B33008F4DECF9EDFAB
:101B5000B091AA00B395B093AA00F894B091A900EF
:101B6000BA95E6E4F0E0EB0FF21D0491789403954A
:101B7000B091AA00B01708F4C6CF88DF87DFB09114
:101B8000A900B395B093A900B091A900BE3008F4A4
:0E1B9000B7CF49DBF89410DFB8E0B1BD77DFC6
:00000001FF
